:100000000C9427020C945F020C945F020C945F0224
:100010000C945F020C945F020C945F020C945F02DC
:100020000C945F020C945F020C945F020C949D226E
:100030000C944C230C94AF1D0C945F020C9483170A
:100040000C945F020C945F020C946E180C94371E93
:100050000C945F020C945F020C945F020C945F029C
:100060000C945F020C945F020C945F020C945F028C
:100070000C945F02200520054C054C05B405D20503
:10008000EA06EA06DD05760687068706DA16DC1636
:10009000E116E416E716EA16ED16B81AAE1ABB1A00
:1000A000031B071B071B031B071B071BDC1A071B74
:1000B000E61AF01A071B071B071B071B031B071B6E
:1000C000071B031B071BC91A071B071B001B001B71
:1000D000001B001B001B001B001B001B001B051B43
:1000E000071BB81AAB1A071B071B071B071B071BAD
:1000F000071B071B071B071B071B051B071B071BF2
:10010000031B071BFE1AFE1AFE1AFE1AFE1AFE1A1F
:10011000FE1AFE1AFE1A051BB923E023D824E02399
:10012000D8242C244F24D824A624B524025114000A
:100130001A000800150017001C0018000C0012001F
:1001400013002A00015104001600070009000A00EC
:100150000B000D000E000F0033002800E100E1004D
:100160001D001B00060019000500110010003600DC
:100170003700E500E000E300E20000002C00000092
:100180002C0000002C003500E7004C0001000100AD
:100190004B00010001002F0030000100520001005F
:1001A0000100010001004A004E004D000100310035
:1001B0003800500051004F00010001000100010013
:1001C0000100010001004600290034000100370051
:1001D0000100010001000100010000000100000019
:1001E00001000000010001000100010001001E00EB
:1001F0001F002000210022002300240025002600EB
:100200002700010001003A003B003C003D003E0099
:100210003F00010001000100010001000100010098
:10022000400041004200430044004500010001003D
:1002300001000100010001000100000001000000B8
:1002400001000000010001000100005C000000004E
:100250000000000000000001010203040506080A76
:100260000C0F1114181C2024292E33393F464C53EF
:100270005B626A7179818A929AA2AAB2B9C1C8CF27
:10028000D5DCE1E7EBF0F4F7FAFCFDFEFFFEFDFC48
:10029000FAF7F4F0EBE7E1DCD5CFC8C1B9B2AAA216
:1002A0009A928A8179716A625B534C463F39332E48
:1002B0002924201C1814110F0C0A08060504030237
:1002C00001010000000000000000000010034500D4
:1002D0007100750069006E006F0078000000260351
:1002E00061006900300033002000440065007300A5
:1002F000690067006E002000530074007500640000
:1003000069006F0000000403090409023B000201B8
:1003100000A0FA09040000010301010009211101F4
:1003200000012240000705810308000109040100C3
:10033000010300000009211101000122B600070598
:100340008203200001120100020000000803A10442
:100350000001000102000105010902A10185020955
:1003600001A1000509190129081500250195087545
:100370000181020501093009311581257F9502753A
:1003800008810609381581257F95017508810605C4
:100390000C0A38021581257F950175088106C0C0B9
:1003A00005010980A101850319012AB7001501265D
:1003B000B700950175108100C0050C0901A10185E8
:1003C0000419012AA002150126A0029501751081C9
:1003D00000C005010906A1018506050719E029E706
:1003E000150025019508750181020507190029EFFF
:1003F0001500250195F075018102050819012905EF
:10040000950575019102950175039101C0050109DA
:1004100006A101050719E029E715002501950875D2
:100420000181029501750881010507190029FF1551
:100430000026FF00950675088100050819012905A9
:10044000950575019102950175039101C000112474
:100450001FBECFEFD4E0DEBFCDBF04B603FE18C091
:100460008091B2029091B302A091B402B091B50212
:100470008730904BA740B04B59F41092B2021092C3
:10048000B3021092B4021092B502E0E0F8E30995CD
:1004900011E0A0E0B1E0E0ECFBE402C005900D92B9
:1004A000AE38B107D9F722E0AEE8B1E001C01D9245
:1004B000A23BB207E1F70E9405130C94DE250C94D1
:1004C000000081E0089581E008950C94630208958E
:1004D0000C9467021F93CF93DF9300D000D01F923C
:1004E000CDB7DEB749835A836B83309191018981FF
:1004F0009A81311114C0662359F0222349F00E94D9
:100500003009182F682F89819A810E94D00803C072
:100510000E940109182F69817A81812F04C00E94ED
:10052000300969817A810F900F900F900F900F9092
:10053000DF91CF911F910C946810FC01262F408110
:1005400051816281738184810C946A0281E00895F3
:10055000CF93DF93EC0160E00E949D02BE01DF912A
:10056000CF910C9468020C94B6110C94B2110895BA
:100570000E947A070E94B7022FEF84E39CE021508B
:1005800080409040E1F700C000000C945D1E0F9386
:100590001F93CF93DF938C0161E00E949D02EC01D9
:1005A000B8010E946502882309F444C0B801CE0155
:1005B0000E94CB168823F1F1B801CE010E94FA1BEC
:1005C0008823C1F1B801CE010E94BE18882391F1A1
:1005D000B801CE010E94561B882361F1F801828187
:1005E000882309F1CB358DE5D807C1F050F4C1154A
:1005F000FCE5DF0781F0CF3DDC45A9F40E94630EE6
:1006000019C0CC35EDE5DE0761F0CD35DD4559F497
:100610000E94A60D08C00E94B8020CC00E94AF0D37
:1006200002C00E94B20DC801DF91CF911F910F91BE
:100630000C94610280E0DF91CF911F910F9108959A
:100640000E94911D80E00E94A7170C943E030E9417
:10065000EF150E9441030C94971D08950C942D03EF
:1006600081E008950C9430030895CF93C82F0E9421
:100670002E038C2F0E943203CF91089580E00C94BA
:1006800035030E94561C0C9435030E94561C909111
:100690009001891721F0809390010C9435030895FF
:1006A000CF93DF93CDB7DEB72B970FB6F894DEBFAD
:1006B0000FBECDBF4F83588769877A878B876111BB
:1006C0000E94F20C9E012F5F3F4F86E0F9011192CC
:1006D0008A95E9F785E0FE013796D90101900D92E0
:1006E0008A95E1F789819A814C815D81452B31F0B2
:1006F0009F3F31F491E08F3F19F403C091E001C0B6
:1007000090E090FF09C049815A816B817C818D8185
:100710009E810E940E0C05C0C9010E94A602811193
:10072000F2CF2B960FB6F894DEBF0FBECDBFDF9190
:10073000CF910895FC01808191810E9472090895F2
:10074000CF93882309F4A9C0C82F8238C1F40E942E
:10075000561C81FDA2C069E38091020190910301C2
:100760000E944C1D0E94140D2FEF81EE94E0215049
:1007700080409040E1F700C0000069E319C0833871
:1007800001F50E94561C80FD88C063E5809102013E
:10079000909103010E944C1D0E94140D2FEF81EED9
:1007A00094E0215080409040E1F700C0000063E5F4
:1007B00080910201909103010E94571DCF910C94EA
:1007C000140D8438C1F40E94561C82FD66C067E493
:1007D00080910201909103010E944C1D0E94140D12
:1007E0002FEF81EE94E0215080409040E1F700C06F
:1007F000000067E4DDCF8CEF8C0F813AF8F48C2F8A
:100800000E940D1B811149C06C2F809102019091B3
:1008100003010E94CC1C882349F06C2F80910201B7
:10082000909103010E94571D0E94140D6C2F80911E
:100830000201909103010E944C1DC0CF80E28C0FF9
:10084000883048F4C77081E001C0880FCA95EAF784
:100850000E94D50CB3CFEBE5EC0FE33040F4F0E0B1
:10086000E75BFE4F808190E0CF910C948A1CE8E515
:10087000EC0FE73150F4F0E0EE0FFF1FE55EFE4FA6
:1008800080819181CF910C94A01CCD3E30F08C2FB3
:100890000E949213CF910C946414CF9108958823F1
:1008A00009F464C0823879F40E94561C81FF5EC04E
:1008B00069E380910201909103010E944C1D0E9406
:1008C000140D69E310C08338B1F40E94561C80FFF8
:1008D0004DC063E580910201909103010E944C1D7F
:1008E0000E94140D63E580910201909103010E9422
:1008F000571D0C94140D843879F40E94561C82FF05
:1009000035C067E480910201909103010E944C1D63
:100910000E94140D67E4E7CF9CEF980F913A10F412
:10092000682FE1CF90E2980F983050F4877091E0F3
:1009300001C0990F8A95EAF7892F0E94DB0CD9CF65
:100940009BE5980F933020F480E090E00C948A1C93
:1009500098E5980F973120F480E090E00C94A01C6B
:100960008D3E20F00E94ED130C94641408951F93A3
:10097000CF93DF93182FEB010E94A003209741F043
:100980008FE99FE00197F1F700C000002197F6CFB3
:10099000812FDF91CF911F910C944F04893319F06F
:1009A00060E070E002C060E570E00C94B70488235A
:1009B00021F00E94D50C0C94140D0895882321F089
:1009C0000E94DB0C0C94140D0895CF92DF92EF92ED
:1009D000FF920F931F93CF93DF937C01D62FC72FE6
:1009E000FC011281058102950F700E94CB0C8823B7
:1009F000B9F01123A9F08C2F807F803421F080E2A0
:100A00008D0F883068F080918F0282FD09C082E0EE
:100A10000E94740D0E94CB0C91E0D82ED92601C003
:100A2000D12CCC2EC2948FE0C8228C2D90E08C303B
:100A3000910508F0CFC1FC01E65CFF4F0C948925BD
:100A40008C2F807FCF70882311F0C295C07F112337
:100A500099F0CC2309F4AAC180E28D0F883010F000
:100A6000D11104C08C2F0E94D50C03C08C2F0E9482
:100A7000E50C0E94140D9AC18D2F0E944F04CC23C7
:100A800009F4A8C180E28D0F883038F1DD2329F107
:100A90008C2F0E94EB0C24C08C2F807FCF70803273
:100AA00011F0C295C07FDD2319F0D130A1F13DC016
:100AB00080918F0282FF17C0112349F0CC2329F0C7
:100AC0008C2F0E94D50C0E94140D80E070C180E034
:100AD0000E944F04CC2309F47DC18C2F0E94DB0CB3
:100AE0000E94140D77C1112371F0002341F00130F1
:100AF00031F40E94F50C8C2B0E94FD0C6BC10E94FE
:100B0000F50C8C2B1DC0002319F0013009F462C1D3
:100B10000E940A0D25C0112321F0063008F05AC1A9
:100B20000EC0053008F056C11BC0112361F0002330
:100B300031F0F701858180FF39C18F7085838C2F5B
:100B40000E94D70447C1002359F0D93309F03FC1AF
:100B5000FFEF07EE13E0F15000401040E1F735C120
:100B60008C2F0E94DE0436C18C2F8695869583706B
:100B700019F0813061F02EC1112321F08D2F9C2FAF
:100B8000937002C080E090E00E948A1C2BC1112368
:100B900021F08D2F9C2F937002C080E090E00E9486
:100BA000A01C20C18D2F112319F00E94921302C0A6
:100BB0000E94ED130E94641415C18C2F837009F0FC
:100BC00047C011110BC12D2F229526952770220F9A
:100BD000220F6D2F6F70862F90E0A0E0B0E0022E04
:100BE00004C0880F991FAA1FBB1F0A94D2F7D4FF15
:100BF00010C04FE050E060E070E004C0440F551FAB
:100C0000661F771F2A95D2F740955095609570958D
:100C100003C040E050E0BA01C695C695C3708A0192
:100C20009B01082B192B2A2B3B2BC901B801C23081
:100C300049F058F4C13019F00E94E607CFC00E9475
:100C4000D407CCC00E94F807C9C00E94D207C6C012
:100C5000112319F08C2F817001C08695882309F427
:100C6000BDC02D2F229526952770220F220F6D2FA4
:100C70006F70862F90E0A0E0B0E0022E04C0880FD5
:100C8000991FAA1FBB1F0A94D2F7D4FF10C04FE0D0
:100C900050E060E070E004C0440F551F661F771FEE
:100CA0002A95D2F7409550956095709503C040E025
:100CB00050E0BA01C695C695C3708A019B01082B06
:100CC000192B2A2B3B2BC901B801C23049F058F42B
:100CD000C13019F00E94AB0881C00E9499087EC003
:100CE0000E94BD087BC00E940C0878C0CF70112301
:100CF00039F08C2F0E9432088D2F0E94D7046EC0CD
:100D00008D2F0E94DE048C2F0E94530867C0D23FB3
:100D100021F128F4D03F41F0D13FC1F043C0D33F8F
:100D200019F1D43F79F03EC0112341F0053008F0AD
:100D300051C08C2F8F710E9478084CC0063008F08B
:100D400049C0F7CF80918F0282FF18C0112339F07C
:100D50008C2F8F710E9432083DC01123C9F38C2F54
:100D60008F710E94530836C0112329F08C2F8F7188
:100D70000E941D082FC00E9418082CC0112349F0A2
:100D8000CF718C2F0E94320863E08C2F0E94590D86
:100D900021C081E00E94740D0230E0F082E00E94E8
:100DA000740D18C0112331F0002391F28D2F0E9491
:100DB000A00310C0002399F2D93349F41FEF27EEA6
:100DC00033E0115020403040E1F700C000008D2F8B
:100DD0000E944F0488EF8C0D843020F40E94561C32
:100DE0000E943503DD20C9F00E94C70C80FD15C0AC
:100DF000F70112820E94C10C0E943208C7010E94B2
:100E00002E070E94C10CDF91CF911F910F91FF908F
:100E1000EF90DF90CF900C945308DF91CF911F910A
:100E20000F91FF90EF90DF90CF9008950F931F9355
:100E3000CF93DF93EC01688179818A810E947D09DB
:100E40008C010E94CF080E94C007B801CE010E9409
:100E5000E504DF91CF911F910F910895CF93DF9318
:100E6000EC01988189812B813C81232B31F08F3FCC
:100E700031F481E09F3F19F403C081E001C080E0BC
:100E800080FD1DC0CE010E94C702811110C00E94CA
:100E9000CB0C8823A1F08A81882389F080918F026E
:100EA00082FD0DC082E0DF91CF910C94740DCE01D4
:100EB0000E941607CE01DF91CF910C94A802DF911A
:100EC000CF91089580E090E00E948A1C80E090E03D
:100ED0000E94A01C0E94F20C0E94140D0E94A315F7
:100EE0000C94641480910201909103010E94621D90
:100EF0000C9462070E94E20C0C94720792959F700A
:100F0000963079F010F4925001C09A50923068F403
:100F1000803F69F018F4883E40F409C0843F29F40A
:100F200006C0883E20F0813F11F080E0089581E006
:100F30000895FC01808191810E9472090E947E07C0
:100F40000895CF93DF9300D000D01F92CDB7DEB7C6
:100F50000F900F900F900F900F90DF91CF91089509
:100F6000CF93DF9300D000D000D0CDB7DEB7269668
:100F70000FB6F894DEBF0FBECDBFDF91CF910895BD
:100F8000089508950C94C1070C94C2070E94C407E9
:100F90006093B4017093B5018093B6019093B7014B
:100FA0000C9462070C94C6070F931F930091B40131
:100FB0001091B5012091B6013091B701602B712BD2
:100FC000822B932B1F910F910C94C6070F931F93A5
:100FD0000091B4011091B5012091B6013091B70193
:100FE00060237123822393231F910F910C94C607D2
:100FF0000F931F930091B4011091B5012091B60198
:101000003091B70160277127822793271F910F9195
:101010000C94C6070C94C1070E940A086093B001A3
:101020007093B1018093B2019093B3010C94620765
:1010300060E070E0CB010C940C080F931F9341E02B
:1010400050E060E070E08A019B0104C0000F111FB6
:10105000221F331F8A95D2F7C901B8011F910F9142
:101060000C940C080F931F9341E050E060E070E097
:1010700004C0440F551F661F771F8A95D2F78091D1
:10108000B0019091B101A091B201B091B3018A0178
:101090009B01082B192B2A2B3B2BC901B8011F914F
:1010A0000F910C940C080F931F9341E050E060E007
:1010B00070E004C0440F551F661F771F8A95D2F752
:1010C00040955095609570958091B0019091B101D7
:1010D000A091B201B091B3018A019B0108231923A9
:1010E0002A233B23C901B8011F910F910C940C08CE
:1010F0000F931F9341E050E060E070E004C0440FA4
:10110000551F661F771F8A95D2F78091B001909185
:10111000B101A091B201B091B3018A019B010827EE
:1011200019272A273B27C901B8011F910F910C9459
:101130000C080F931F930091B0011091B101209101
:10114000B2013091B301602B712B822B932B1F9135
:101150000F910C940C080F931F930091B001109104
:10116000B1012091B2013091B30160237123822338
:1011700093231F910F910C940C080F931F930091D0
:10118000B0011091B1012091B2013091B3016027FB
:101190007127822793271F910F910C940C080895B3
:1011A000282F362F892F6CE00E940C25820F982F54
:1011B0009770A1E001C0AA0F9A95EAF786958695E7
:1011C000869590E065E070E00E941525FC01EE56E2
:1011D000FE4F40E050E0632F70E090819B01042EB1
:1011E00002C0369527950A94E2F7217021952927A8
:1011F0002A23292721934F5F5F4F4530510569F717
:101200000895282F892F6CE00E940C25820FA82FAB
:10121000A77086958695869590E065E070E00E94BF
:101220001525BC0140E050E080E0FB01E40FF51F14
:10123000EE56FE4F208130E00A2E02C036952795EB
:101240000A94E2F721703327042E01C0220F0A947A
:10125000EAF7822B4F5F5F4F4530510531F7089514
:10126000BF92CF92DF92EF92FF920F931F93CF9393
:10127000DF938C01C090B001D090B101E090B20139
:10128000F090B3018091B4019091B501A091B601A5
:10129000B091B701C82AD92AEA2AFB2ACFE1D0E0C7
:1012A000D701C6010C2E04C0B695A79597958795D2
:1012B0000A94D2F780FD04C0219790F7B12C07C0A3
:1012C000BC2EB8018C2F0E9483100197A9F38B2D9F
:1012D000DF91CF911F910F91FF90EF90DF90CF9012
:1012E000BF900895CF93DF93EC010E943009BE01B7
:1012F0000E948310DF91CF9108951F93CF93DF93C6
:10130000EB0190919101992321F0CB010E94720988
:1013100013C0882349F0CB010E943009182F682F91
:10132000CE010E94D00804C0CB010E940109182FF1
:10133000BE01812F0E948310DF91CF911F910895EC
:10134000CF93DF93C091B8018091B901C817A1F084
:10135000D0E0CE0166E070E00E941525FC01E65465
:10136000FE4F4081518162817381848195810E9409
:10137000B0072196C770E8CFDF91CF9108954091D3
:10138000EA015091EB016091EC017091ED018091C7
:10139000EE019091EF010C94B007FF920F931F9311
:1013A000CF93DF938091EF0182958F7009F062C037
:1013B0008091EC01882309F45DC02091B801F09080
:1013C000B9011091EA010091EB01A091ED01B091FA
:1013D000EE0181E01F3F09F080E0C0910001D09153
:1013E0000101482F2F1509F445C0109721F00F3F38
:1013F00021F080E003C081E001C0842F30E080FD57
:1014000035C0C90166E070E00E941525FC01E65474
:10141000FE4F818180132AC08081811327C0828181
:10142000811124C0838194818A1B9B0B8C179D079B
:10143000E8F48091EF018F7080618093EF01C90122
:1014400066E070E00E941525FC01E154FE4F90819A
:101450009F70906190838AEE91E00E942E07DF9149
:10146000CF911F910F91FF900C94A0092F5F3F4FD8
:101470002770B8CFDF91CF911F910F91FF90089502
:101480009F92AF92BF92CF92DF92EF92FF920F9313
:101490001F93CF93DF93CDB7DEB761970FB6F89464
:1014A000DEBF0FBECDBF8C0185E0F801DE011D96C9
:1014B00001900D928A95E1F7F801E2809091EA019E
:1014C0003091EB016091ED017091EE0161157105B4
:1014D00031F03F3F31F481E09F3F19F403C081E0D8
:1014E00001C080E0F82FF1709F2E80FD47C1F80108
:1014F00040812181A380B4808AEEC82E81E0D82E5D
:10150000F090EC01F501E61BF70B60910001709182
:101510000101FF2009F4DCC08091EF01582F507FBA
:10152000E617F70708F096C0511155C0231313C0F2
:10153000491311C0FE2CE1100EC08F7080618093A2
:10154000EF010E94BF09C6010E942E078091EF01A2
:10155000F801858350C1AB2831F02F3F31F481E091
:101560004F3F19F403C081E001C080E080FD03C05B
:1015700081E08E2502C080E090E0F82FF170FF2E10
:1015800080FF1FC0E091B8013091B901E31709F461
:1015900010C1F0E0CF0166E070E00E941525DC018B
:1015A000A654BE4F11968C911197281307C08C91A9
:1015B000481304C012968C91E81203C03196E7706C
:1015C000E5CFFE2CEE2009F416C18091EF01816079
:1015D0008093EF0154C0231306C0491304C0E110E7
:1015E00002C0F80199C0C8010E949907882361F1DF
:1015F000EE2051F12091EF01822F82958F7090E0C3
:10160000029774F08091EA019091EB0198878F83A3
:101610001986BB86AA862C87CE0107960E942E07C4
:1016200086E0F801AAEEB1E001900D928A95E1F70B
:101630000E94CD090E94BF090AC0231711F1C801F9
:101640000E94990781112CC0C8010E942E07FF2417
:10165000F394D1C05111F1CF7A2DB98AA88A522FB3
:101660006E2D89890E94A1078AEE91E00E942E07C3
:1016700086E0F60111928A95E9F70E94BF09F12CE4
:10168000BAC04913DCCFE110DACFF8018583C80175
:101690000E942E0786E0F60111928A95E9F7ABC009
:1016A000EE2091F22091EF01822F82958F7090E0D1
:1016B00002970CF4B5CF8091EA019091EB019A83E7
:1016C00089831B82BD82AC822E83CE010196A6CF78
:1016D000E617F70708F044C0FE2CEE2009F4B4CF5B
:1016E000231330C049132EC02091EF0120FD21C0EB
:1016F000822F82958F70482F50E041155105C9F017
:10170000F80125834F30510541F08F5F982F929556
:10171000907F822F8F70892B8583C8010E942E07AE
:1017200086E0F801AAEEB1E001900D928A95E1F70A
:101730003DC086E0F801AAEEB1E001900D928A95D5
:10174000E1F759C0C8010E949907811169CF8091C2
:10175000EF0181608093EF01C8010E942E074BC00A
:101760007A2DB98AA88A522F6E2D89890E94A107E5
:1017700086E0F60111928A95E9F718C0EE2009F487
:1017800063CFC8010E949907F82E882309F45CCF23
:1017900086E0F801AAEEB1E001900D928A95E1F79A
:1017A0008AEE91E00E949A030E94CD090E94BF092F
:1017B00022C04D872E878D859E850E947209292F14
:1017C00022952F70223028F49F7039F0811105C0C6
:1017D0000BC0243028F49F7049F4805E883020F0DC
:1017E000C8010E942E079F2CF92C05C0F801958195
:1017F000907F99F7F9CF8F2D61960FB6F894DEBFE1
:101800000FBECDBFDF91CF911F910F91FF90EF9051
:10181000DF90CF90BF90AF909F900895CF93DF93CC
:10182000CDB7DEB72C970FB6F894DEBF0FBECDBF95
:101830004F83588769877A878B879C87CE01079665
:101840000E94400A8823D1F09F8188852A853B85A4
:10185000232B31F08F3F31F481E09F3F19F403C017
:1018600081E001C080E080FD6FC04F8158856985AF
:101870007A858B859C850E94B00766C086E0FE0154
:101880003796DE01119601900D928A95E1F7FF815E
:10189000E8856A857B856115710531F0EF3F31F48C
:1018A00081E0FF3F19F403C081E001C080E080FDCA
:1018B0004BC08091B90190E09C012F5F3F4F277092
:1018C00033274091B80150E02417350709F443C08D
:1018D000F983EA837D836C8366E070E00E941525BE
:1018E000DC01A654BE4F96E0FE01319601900D92A8
:1018F0009A95E1F72093B9010E94A00925C090E0D4
:1019000066E070E00E94152586549E4F0E94400AB2
:10191000882371F18091B80190E066E070E00E9448
:101920001525FC01E654FE4F40815181628173818F
:10193000848195810E94B0078091B80190E0019662
:10194000877099278093B8018091B8019091B9016F
:101950008913D5CF0DC00E947A071092B901109259
:10196000B801EAEEF1E086E0DF011D928A95E9F721
:101970002C960FB6F894DEBF0FBECDBFDF91CF918E
:10198000089580911002859585958595089580919B
:1019900010028770089590911002977081E009F409
:1019A00080E0089580913302089590913302892B4D
:1019B0008093330208958095909133028923809318
:1019C0003302089510923302089590913202892BC8
:1019D00080933202089580959091320289238093FA
:1019E00032020895109232020895809111020895F2
:1019F00008950C94F80C0C94F90C90918F0292FDC0
:101A000008C090911102981721F0809311020C9454
:101A1000FB0C089580911102882329F01092110285
:101A200080E00C94FB0C0895CF93DF93E0910201CA
:101A3000F0910301809133028083E0910201F091E3
:101A40000301908180913202892B80838091110261
:101A5000882381F0E0910201F09103019081892BAC
:101A6000808380910201909103010E94B61C811134
:101A70000E940A0DC0910201D091030140E250E0A2
:101A800060EF71E0CE010E948F25892B69F080E222
:101A9000FE01A0EFB1E001900D928A95E1F7CE0131
:101AA000DF91CF910C94621CDF91CF9108950C943B
:101AB000F80C90918F0292FD10C0982F990F990FFA
:101AC000990F692B609310020E94320880911002D6
:101AD0008595859585950C94570D0C943208109238
:101AE000100280E00C94570D209110028095822303
:101AF00080931002982F977099F430E0482F082EA9
:101B0000000C550B2417350759F090918F0292FD68
:101B100007C08595859585950E9453080C946F0D97
:101B2000089590918F0292FB222720F9281769F0DF
:101B300080FB92F990938F0280918E0290918F0298
:101B40000E94DF0D82E00C94740D089580918F0245
:101B500082FB882780F991E089270C94910D81E020
:101B60000C94910D80E00C94910D6FEF7FEF80E06D
:101B700090E00C94C82580E090E00E94A42521E02C
:101B8000893E9E4F09F020E0822F089582E090E088
:101B90000C949C2583E090E00C949C25CF9384E0EA
:101BA00090E00E949C25C82F82E290E00E949C2534
:101BB0002C2F30E0A901582BCA01CF910895CF9363
:101BC000C92F682F84E090E00E94AA256C2F82E242
:101BD00090E0CF910C94AA25AB01BC018FE090E07E
:101BE0000C94BC25AB01BC0183E190E00C94BC25B6
:101BF00060E070E0CB010C94F20D60E070E0CB018E
:101C00000E94EC0D0C94F80D69EE7EEF80E090E000
:101C10000E94C82560E082E090E00E94AA2560E072
:101C200083E090E00E94AA251092B4011092B501C1
:101C30001092B6011092B70160E084E090E00E943B
:101C4000AA2560E082E290E00E94AA2560E085E09B
:101C500090E00E94AA2560E086E090E00E94AA251C
:101C60006FEF87E090E00E94AA2540E050E0BA01C3
:101C700088E090E00E94BC2560E08DE090E00E944A
:101C8000AA2540E050E0BA0188E190E00E94BC251E
:101C900060E087E190E00E94AA2540E050E0BA01B0
:101CA0008CE190E00E94BC2560E070E080E290E072
:101CB0000E94C82540E050E0BA0188E190E00E940F
:101CC000BC250C94FD0D0C94040E682F8EE090E062
:101CD0000C94AA250E941C1E60934002709341023E
:101CE000809342029093430260933C0270933D02C2
:101CF00080933E0290933F02089581E008950C94F2
:101D00007D0E08950C94810E0C94810E0C94840E1B
:101D10000C94810E0C94880E0C94810E8FE591E149
:101D20000E944C1C0E948C0E0C948A0E0E94820E03
:101D30000C94810E0E9479110E9434030C94A8180F
:101D40000E94071E0E945E120E949A0E0E94EF15CA
:101D50000C94860E5F926F927F928F929F92AF92B9
:101D6000BF92CF92DF92EF92FF920F931F93CF9388
:101D7000DF93CDB7DEB72A970FB6F894DEBF0FBE5C
:101D8000CDBF0E947312C82E81110E946A0E34E3E7
:101D9000832E32E0932E00E010E0502E802F0E9420
:101DA0009D115C01F401619071904F0168267926C4
:101DB00061147104B1F40F5F1F4F0430110569F70E
:101DC0008FEF89838A831B820E94101E8160782F87
:101DD0009D838C8349815A816B818D810E94500340
:101DE0003AC08091440281FD0E94A611D12CEE24BC
:101DF000E394F12CC3018E219F21892B29F10E94AC
:101E00007F0E8823A9F0DE825F82AE20BF2081E0B2
:101E1000AB2809F480E088870E94101E8160782F2B
:101E20009A8789874E815F8168858A850E945003E1
:101E3000000F111FF801EC5CFD4F80819181E826B5
:101E4000F926F182E08207C0D394EE0CFF1CFCE07F
:101E5000DF12D0CFB0CF81E0C11001C080E02A9660
:101E60000FB6F894DEBF0FBECDBFDF91CF911F91AB
:101E70000F91FF90EF90DF90CF90BF90AF909F9029
:101E80008F907F906F905F9008950E94AA0E0E949D
:101E9000F3170E9482140C944503CF93DF930E94A2
:101EA0008810EC01811521E5920708F045C08115E5
:101EB00030E5930708F094C0883E910528F5803EF0
:101EC000910508F001C1883A910570F4853A9105B1
:101ED00008F07CC08130910509F475C008F4F1C0A8
:101EE000049708F0F1C0EDC08F3B910508F0E9C000
:101EF000C85AD0E0CC0FDD1FC45BDE4F0990D881FB
:101F0000C02DCE019464E1C0811540E2940758F4DD
:101F1000811551E0950708F0D7C08D3E910508F472
:101F2000D0C09065D2C0C11580E4D80708F4C9C0FC
:101F3000DF70CE01906AC9C0811525E59207A8F42B
:101F4000811534E5930708F09EC0811543E5940799
:101F500008F081C0811552E5950708F064C0D82FBC
:101F6000CC27CE01816F906AB0C0C11589E5D80732
:101F7000A0F4C11528E5D20708F08BC0C11536E5DD
:101F8000D30708F09EC08C2F0E941C118F7190E027
:101F9000D82FCC27CE01906298C0C1154AE5D4074E
:101FA00008F47DC0CE0190568115904208F089C09A
:101FB0008D2F8F710E941C11DD27D0628F71AE01B1
:101FC000582BCA0182C081E090E07FC0C55AD0E0A2
:101FD000C658DE4F8881C82FD0E0CE01906475C00E
:101FE000F4E096958795FA95E1F7282F23703C2F1A
:101FF000337081E090E002C0880F991F3A95E2F7B4
:102000009C68AC01522B9C2F9F7096959695892FBA
:1020100090E0EC01A5E0CC0FDD1FAA95E1F7CA0125
:102020008C2B9D2B52C08370992721E030E002C099
:10203000220F331F8A95E2F79C2F96959695C92F0C
:10204000D0E075E0CC0FDD1F7A95E1F7C22BD32BE2
:10205000CE019C683AC08370992721E030E002C02D
:10206000220F331F8A95E2F79C2F96959695C92FDC
:10207000D0E065E0CC0FDD1F6A95E1F7C22BD32BD2
:10208000CE019A6822C0D82FCC27CE01846F906AE7
:102090001CC0DC2FCC27CE01806F906A16C08C2F1D
:1020A0008F700E941C1194E0D695C7959A95E1F720
:1020B000CF70D0E0DC2FCC27D0699E01282BC9013E
:1020C00004C080E090E001C0CE01DF91CF9108957F
:1020D000382F262F872F90E06CE070E00E941525A6
:1020E000FC01832F90E060E370E00E9415258E0FC5
:1020F0009F1FFC01E20FF11DEE0FFF1FE45DFE4F7D
:102100008591949108950E9468100E944D0F089542
:102110008238910569F1B0F48133910509F46DC0FD
:1021200048F48932910509F463C08A32910509F4B3
:1021300069C008958533910509F455C08933910527
:10214000B9F00895833E910569F138F4803E910518
:10215000B1F0823E910509F10895863E9105A9F1FD
:10216000873E9105B9F1843E910509F064C023C012
:1021700020918E0220FD4FC021FD4DC00895809119
:102180008E0280FD44C080918F0280FF44C0809108
:102190008E0284FD42C083EE4DC080918E0282FF8C
:1021A00038C0F5CF80918E0282FD33C080918F02BE
:1021B00080FD31C0ECCF80918F0281FF32C08091D1
:1021C0008E0284FD2AC087EE35C080918E0283FF87
:1021D00026C0F5CF80918E0283FD21C080918F02B1
:1021E00081FD1FC0ECCF80918E0285FD1CC01DC0FB
:1021F00080918E0285FD19C016C080918E0286FDE9
:1022000016C017C080918E0286FD13C010C089E3EE
:1022100011C082EE0FC080EE0DC080E00BC086EED4
:1022200009C084EE07C089E205C085E303C08AE2E5
:1022300001C081E390E0089590918E0292FF0DC05D
:10224000282F2871283019F4877F846006C0282F32
:102250002471243011F48B7F886093FF0DC0282FE8
:102260002871283119F4877E846106C0282F2471D3
:10227000243111F48B7E886120918F0220FF0DC0E4
:10228000382F3871383019F4877F816006C0382FB5
:102290003171313011F48E7F886021FF0DC0282FFD
:1022A0002871283119F4877E816106C0282F217199
:1022B000213111F48E7E886194FD877E089580E03F
:1022C00008950C94B50D0E9473128FE39CE9019759
:1022D000F1F700C000000E94731280E00E949D117F
:1022E00080FF04C00E9461110C945D1E08950C943F
:1022F00063110E94BB0D811102C00E94630E0E94F7
:10230000C60D809344020E94CE0D90938F0280935D
:102310008E020E9477110E94CA0D682F70E080E043
:1023200090E00E94D2076091B0017091B10180915C
:10233000B2019091B3010C940A08E82FF0E0EE0F7F
:10234000FF1FE856FD4F808191810895089580EA2E
:102350008A95F1F7089500C008950C94A711089587
:102360000C94AF110C94B0110C94AF110C94B411E7
:10237000F894E82FE295EF70F0E031A1282F2F704C
:1023800081E090E001C0880F2A95EAF7982F909598
:10239000932391A392A1892B82A3789408950F93FC
:1023A0001F93CF93DF93C9E8D1E089918F3F11F05C
:1023B0000E94B81181E0CD38D807B9F7CDE7D1E058
:1023C00009E811E089918F3F11F00E94B8110C17B4
:1023D0001D07C1F7DF91CF911F910F910895BF9213
:1023E000CF92DF92EF92FF920F931F93CF93DF93E1
:1023F0008C01C62FD0E0CE0187579E4F6C01FC01A7
:1024000090819F3F09F450C0B62EF894E92FE295D1
:10241000EF70F0E081A19F7021E030E001C0220F59
:102420009A95EAF7822B81A382A12095282322A3E3
:1024300078940E94AB11EDE7F1E049E851E021E02A
:1024400030E0E12CF12C61916F3F89F0A62FA2952D
:10245000AF70B0E090968C9190E06F7002C095954F
:1024600087956A95E2F780FD02C0C90102C080E04D
:1024700090E0E82AF92A220F331F4E175F0719F759
:10248000F60180818F3F11F00E94B81161E0E114E4
:10249000F10409F460E08B2D0E94AD11CC0FDD1F1B
:1024A000C00FD11FF982E882DF91CF911F910F9168
:1024B000FF90EF90DF90CF90BF9008950E94CF11D2
:1024C00088E0E8E9F2E0DF01982F1D929A95E9F79C
:1024D000E0E9F2E0DF011D928A95E9F784E00E94CD
:1024E000BE120C94B302FF920F931F93CF93DF930E
:1024F000CDB7DEB728970FB6F894DEBF0FBECDBFBD
:102500008E010F5F1F4F88E0F80111928A95E9F75D
:10251000F12C6F2DC8010E94EF11F394F4E0FF122B
:10252000F8CF48E050E0B80180E992E00E948F25A2
:10253000FF24F394009709F4F12C892B41F088E0F3
:10254000F801A0E9B2E001900D928A95E1F72F2DF4
:1025500044E068E972E080E992E00E94BF120E94C4
:10256000B5028F2D28960FB6F894DEBF0FBECDBFF3
:10257000DF91CF911F910F91FF9008950895FF92E1
:102580000F931F93CF93DF93F82E092F162FD72F7A
:10259000C42F222349F081E0809347020E94101E3D
:1025A0009093460280934502809147028823D9F098
:1025B00080914502909146020E94281E059798F04E
:1025C000EF2DF02FA12FBD2F80E090E04C2F50E099
:1025D0008417950734F4219131912D933D93019601
:1025E000F7CF10924702DF91CF911F910F91FF908B
:1025F00008950E9413200E94A00E0C941F200E9498
:1026000023200E94450F0C943D200E94AE1D0E9485
:10261000FA1F0E948E0E0E94F9120E94FF120E9461
:10262000960EFBCF80914E0280FF06C0609109019B
:1026300070E0660F771F2CC081FF08C06091090110
:1026400070E0660F771F660F771F22C082FF09C0F8
:102650006091090170E043E0660F771F4A95E1F74A
:1026600017C060914D026623D1F0209108016217D6
:1026700078F78091090190E070E033E0880F991FAE
:102680003A95E1F70E941525622F70E00E945325CC
:102690006038710540F46115710519F406C068E0F1
:1026A00070E0862F08958FE7089581E00895809166
:1026B0004E0280FF08C06091050170E07595679536
:1026C0007595679523C081FF06C06091050170E094
:1026D000759567951BC082FF04C06091050170E08D
:1026E00012C060914C026623A9F020910401621788
:1026F000A0F78091050170E090E00E941525622FFF
:1027000070E00E9453256038710540F46115710531
:1027100019F406C061E070E0862F08958FE70895F0
:1027200081E008958D3E21F40E941213819504C02A
:102730008E3E29F40E9412138093520208958F3E18
:1027400021F40E941213819504C0803F29F40E9455
:102750001213809351020895893F19F40E94571370
:1027600005C08A3F31F40E9457138195809353022C
:1027700008958B3F21F40E945713819504C08C3F2C
:1027800029F40E9457138093540208959FE0980FF4
:10279000983078F421E030E0A90102C0440F551FC1
:1027A0009A95E2F7CA0190915002892B80935002CA
:1027B00008958D3F21F480914E0281600BC08E3FC1
:1027C00021F480914E02826005C08F3F29F48091F0
:1027D0004E02846080934E0208958D3E39F49091AC
:1027E000520297FF35C01092520259C08E3E29F412
:1027F000909152021916BCF32BC0909151028F3E5A
:1028000029F497FF25C01092510249C0803F19F466
:102810001916CCF31DC090915302893F29F4191663
:10282000BCF4109253023BC08A3F19F497FF10C0CA
:10283000F8CF8B3F39F49091540297FF09C0109262
:1028400054022DC08C3F21F4909154021916BCF310
:102850009FE0980F983080F421E030E0A90102C099
:10286000440F551F9A95E2F7CA0180959091500246
:1028700089238093500213C08D3F21F480914E0232
:102880008E7F0BC08E3F21F480914E028D7F05C05C
:102890008F3F29F480914E028B7F80934E0280916E
:1028A0005102811106C080915202811102C0109222
:1028B0004D0280915302811106C080915402811112
:1028C00002C010924C0208950E94101E20915102E5
:1028D000211104C020915202222321F090934B0237
:1028E00080934A0220915302211104C02091540286
:1028F000222321F090934902809348028FE492E0D2
:102900000C947C1CEF92FF920F931F93CF93DF9355
:1029100000D000D000D0CDB7DEB786E0EFE4F2E023
:10292000DE01119601900D928A95E1F7E090510237
:10293000F0905202009153021091540210925102F1
:10294000109252021092530210925402E11003C0EE
:10295000FF2009F464C080914A0290914B020E94CA
:10296000281EFC0120914D02222339F080910A019A
:1029700090E08E179F0760F052C080910B0190E0AD
:102980006AE070E00E9415258E179F0718F047C077
:102990002F3F19F02F5F20934D02EE2061F00E942F
:1029A0001213682F1E1414F08FEF01C081E00E94F3
:1029B0000C2580935102FF2061F00E941213682FB2
:1029C0001F1414F08FEF01C081E00E940C2580934A
:1029D000520280915102882311F120915202222348
:1029E000F1F0082E000C990B65EB70E00E941525A4
:1029F000992319F09093510203C081E08093510212
:102A0000822F220F990B65EB70E00E941525992308
:102A100019F09093520203C081E080935202011199
:102A200003C0112309F464C08091480290914902C7
:102A30000E94281EFC0120914C02222339F0809133
:102A4000060190E08E179F0760F052C08091070149
:102A500090E06AE070E00E9415258E179F0718F03D
:102A600047C02F3F19F02F5F20934C02002361F0E5
:102A70000E945713682F101614F08FEF01C081E0E9
:102A80000E940C2580935302112361F00E9457137A
:102A9000682F111614F08FEF01C081E00E940C2501
:102AA0008093540280915302882311F120915402A3
:102AB0002223F1F0082E000C990B65EB70E00E94C8
:102AC0001525992319F09093530203C081E0809358
:102AD0005302822F220F990B65EB70E00E9415259F
:102AE000992319F09093540203C081E0809354021B
:102AF0008091510281110BC080915202811107C057
:102B000080915302811103C08091540281110E946F
:102B10006414EB82FC820D831E8386E0FE013196F5
:102B2000AFE4B2E001900D928A95E1F726960FB6D8
:102B3000F894DEBF0FBECDBFDF91CF911F910F91F3
:102B4000FF90EF900895EFE4F2E086E0DF011D9240
:102B50008A95E9F710924D0210924C0210924E02A3
:102B6000089586E090E00C949C25682F86E090E024
:102B70000C94AA258091A002847089628093A0029F
:102B80000C94B5158091A00286958695869508953A
:102B90008091A00281FD07C082608093A0020E9404
:102BA000B5150C94F41708958091A00281FF07C019
:102BB0008D7F8093A0020E94B5150C94FE17089596
:102BC0008091A00281FD0C94D4150C94C8158091BD
:102BD000A00286958170089580910C0108950E944D
:102BE000BB0D811104C00E94630E0E94BA150E94A1
:102BF000B1158093A002282F26952695269530E0C2
:102C00002630310524F0877088628093A00280917D
:102C1000A00280FF04C086958695869501C080E05D
:102C20000C94A7172091A002822F869586958695F1
:102C3000482F50E04530510554F48F5F982F990F7D
:102C4000990F990F822F8770892B8093A002809112
:102C5000A00281608093A0020E94B5158091A0021D
:102C60008695869586950C94A7178091A002982F3B
:102C7000969596959695A1F0915E990F990F990F5B
:102C80008770892B8093A002887F91E009F490E0FF
:102C90008091A00290FB80F98093A0020E94B5155C
:102CA0008091A0028695869586950C94A7178091B1
:102CB000A00280FD13C081608093A002813019F4CE
:102CC00089E08093A0028091A0020E94B5158091B6
:102CD000A0028695869586950C94A71708958091F5
:102CE000A00280FF08C08E7F8093A0020E94B515CD
:102CF00080E00C94A71708958091A00280FD0C94A9
:102D00006F160C9457169091A002892F8695869580
:102D100086958F5F8F719770863038F4880F880F93
:102D2000880F892B8093A00202C09093A00280910B
:102D3000A002887F91E009F490E08091A00290FBCE
:102D400080F98093A0020E94B5158091A00286951B
:102D5000869586950C94A717863008F085E09091AB
:102D6000A0029770282F220F220F220F922B9093F0
:102D7000A002987F21E009F420E09091A00220FBBE
:102D800090F99093A0020C94A7170E94AC16809122
:102D9000A0020C94B515FC01DB0112968C918823DE
:102DA000F9F0EC5BFC45E730F105D8F4EA5BFF4F46
:102DB0000C94892585E001C080E00E94C51680E062
:102DC00008950E943516FBCF0E941216F8CF0E947C
:102DD0007C16F5CF0E948316F2CF0E94E015EFCF4C
:102DE00081E00895519A59980895599A08955998EB
:102DF00008958F929F92AF92BF92CF92DF92EF92FF
:102E0000FF920F931F93CF93DF938C0180918600E5
:102E1000909187006CE070E00E943F256017710779
:102E200030F0C80169E070E00E943F255EC08091EB
:102E3000860090918700E0908600F0908700E091F6
:102E40008600F0918700C6E0D0E0BE010E943F25D9
:102E500020E030E0060F171F211D311D48015901E8
:102E600085E0880C991CAA1CBB1C8A95D1F7C70168
:102E7000BE010E943F256F01E12CF12CA7019601B4
:102E8000260F371F411D511DC501B4010E94672542
:102E900069017A01C0918600D0918700CA01B90109
:102EA0000E9426259E0140E050E00E942625A701B1
:102EB00096010E942625DC01CB012FE0B695A7954F
:102EC000979587952A95D1F70091860010918700F4
:102ED00020E030E0081719072A073B0728F4609123
:102EE000860070918700CB01BC01CB01DF91CF91AF
:102EF0001F910F91FF90EF90DF90CF90BF90AF9018
:102F00009F908F9008951F920F920FB60F921124E9
:102F10002F933F934F935F936F937F938F939F93E1
:102F2000AF93BF93EF93FF930E94F716FF91EF913A
:102F3000BF91AF919F918F917F916F915F914F91D1
:102F40003F912F910F900FBE0F901F901895CF9328
:102F5000C82F8630A8F4811114C080918800909108
:102F60008900892B51F080916F008D7F80936F00D5
:102F700080916F008E7F80936F000E94F71611C0C2
:102F8000C5E08091880090918900892B51F480914F
:102F90006F00826080936F0080916F0081608093EA
:102FA0006F00609186007091870080E090E02C2F88
:102FB00030E040E050E00E94262525E030E040E08F
:102FC00050E00E946725B42FA32F922F8827892FC6
:102FD0009A2FAB2FBB270E94F916909389008093FC
:102FE0008800CF91089508951092570210925602CA
:102FF0001092580281E08093550208951092550274
:103000000E94C2150C94A7170F931F93CF93DF93C1
:1030100080910D0191E0980F823019F090930D018D
:1030200058C081E080930D010E94EC15182FC091CB
:103030005602D091570221960E94EC1590E068E765
:1030400070E00E941525BC01CE010E943F259C0125
:103050009093570280935602812F90E068E770E0CA
:103060000E941525BC01660F672F661F770B7195AF
:10307000C9010E943F256F7780915802823019F470
:10308000603439F404C0813021F46F3711F41092A8
:103090005502E62FF0E0E45BFD4FC49100918600FD
:1030A000109187000E94C215282F8C2F90E0B80144
:1030B0000E9415256BEF74E00E943F25CB01622F23
:1030C00070E00E9415250E94F91690938900809364
:1030D0008800DF91CF911F910F9108951F920F9259
:1030E0000FB60F9211242F933F934F935F936F93DB
:1030F0007F938F939F93AF93BF93EF93FF938091B1
:10310000550281110E940418209188003091890095
:1031100080918600909187006AEF70E00E943F25C1
:103120006B5F7F4F6217730710F40E94F516FF91D3
:10313000EF91BF91AF919F918F917F916F915F912F
:103140004F913F912F910F900FBE0F901F901895A8
:103150000E94F21682E08093800089E180938100D2
:103160008FEF9FEF90938700809386000E94EF156A
:103170000E94E71581110C94F4170895CF93DF9303
:10318000EC01FB018281882309F43CC1C430FDE5D8
:10319000DF0760F4CB3F9CE5D90788F49E012250FD
:1031A0003C452431310508F02EC109C0C236EDE599
:1031B000DE0729F0C63AFDE5DF0709F024C10E94C9
:1031C000CE0D90938F0280938E02C1318CE5D8078B
:1031D00009F4C6C008F042C0C930ECE5DE0709F4C6
:1031E0009BC000F5C5308CE5D80709F485C078F49C
:1031F000C330ECE5DE0709F478C008F07AC0C230CD
:10320000DC4509F0F5C080918E028160EFC0C730C7
:103210009CE5D90709F478C008F07AC080918E0245
:103220008061E4C0CD30FCE5DF0709F487C058F4C5
:10323000CB309CE5D90709F479C008F07BC08091B8
:103240008E0288606FC0CF30FCE5DF0709F480C0D4
:1032500008F082C080918E02877FC8C0CE3F9CE577
:10326000D90709F471C000F5C531FCE5DF0709F4A1
:1032700085C068F4C3319CE5D90709F475C008F02E
:1032800095C00E947A0780918E028F77AFC0CC3FA5
:10329000FCE5DF07A9F108F054C0CB3FDC4509F09D
:1032A000A7C080918F0240C0C230EDE5DE0709F46F
:1032B00089C058F4C1158DE5D80709F45AC008F043
:1032C00069C080918F0282602FC0C236EDE5DE07B3
:1032D00009F47CC0C63AFDE5DF0709F481C0C330BC
:1032E000DD4509F085C080E06EC080918E0282606D
:1032F0007DC080918E0216C080918E02886076C05B
:1033000080918F0282604FC080918E0280626EC079
:1033100080918E0280646AC00E947A0780918E023A
:10332000806864C0846062C081603DC080918E020C
:103330008E7F5CC080918E028D7F58C080918E02FE
:1033400016C080918F0218C080918F028D7F2BC094
:1033500080918E028F7E4AC080918E028F7D46C002
:1033600080918E028F7B42C080918E02877F8B7FFF
:103370003DC080918F028D7F8E7F15C080918E021F
:1033800082FB222720F991E0922790FB82F990FBA3
:1033900083F92CC080918F02982F909591708E7F29
:1033A000892B90FB81F980938F0222C00E947A07BB
:1033B00080918E0287FB222720F991E0922790FBD3
:1033C00087F914C081E00E94650E12C080918E02C0
:1033D00084FB222720F991E0922790FB84F906C014
:1033E00080918E02982F909590FB80F980938E02A9
:1033F00080918E0290918F020E94DF0D0E947A07C9
:1034000080E001C081E0DF91CF910895893289F198
:10341000F0F4843171F1B0F4873009F077C081E0C5
:1034200080930B0184E180930A018AE08093090173
:103430008EE18093080188E08093050188E2809303
:10344000040164C092EE980F9A30F0F05FC08035AE
:1034500009F444C028F48F3409F058C08AE03FC012
:10346000813529F0823509F051C081E038C08FEFF5
:1034700036C080915B02882379F110925B02109232
:103480005A021092590242C08D5180935B028330E0
:1034900099F038F4813069F08230D9F48AE091E013
:1034A0000DC0853099F078F0863099F484E091E091
:1034B00005C08BE091E002C089E091E090935A0250
:1034C0008093590223C088E091E0F8CF85E091E035
:1034D000F5CF10925B021AC080E0089586EFE0916C
:1034E0005902F0915A02309789F02081082E000C81
:1034F000990B820F911D8F3F910519F014F08FEFFA
:1035000004C097FF02C0108201C0808381E008954B
:103510000F931F9341E050E060E070E08A019B014F
:1035200004C0000F111F221F331F8A95D2F7C90153
:10353000B8010E94D2071F910F910C947A07482F6F
:1035400050E0FA013597EF33F10508F060C0E35B16
:10355000FF4F0C9489250E94630E55C08091440250
:10356000817F8E7F8093440281E080935C02089586
:103570000E94B80248C080914402982F90959170A3
:1035800090FB80F98093440291113DC0897F877F31
:1035900010C08091440281FB222720F991E09227FC
:1035A00090FB81F980934402992369F18091440250
:1035B00081608093440227C08091440282FB2227CD
:1035C00020F991E0922790FB82F9ECCF80914402A0
:1035D00083FB222720F991E0922790FB83F9E2CF29
:1035E0000E947A0780918E0287FB222720F991E0C2
:1035F000922790FB87F980938E0205C0895301C002
:103600008D510E94881A81E0089580E0FACF80E011
:10361000089580E008950C94091BCF93C82F8091E2
:103620005C02813069F038F08230C1F58C2F0E9445
:10363000061A81E039C00E94D20C823289F504C09A
:103640000E94D20C823261F48C2F0E940B1B8111DC
:1036500004C08C2F0E949F1A1FC081E090E01CC004
:103660008C2F0E94091B811116C0C43189F058F4B7
:10367000CB3089F0C031B1F482E080935C0288E302
:103680000E94061A08C0C93219F0C83321F00AC0D6
:1036900010925C0207C081E0817006C010925C024B
:1036A00080E002C080E0F8CFCF910895CF93DF9300
:1036B00086319C4541F5EB010E94D20C982F8A81FE
:1036C0002091020130910301882379F09A7A81E0F8
:1036D00009F480E080935D02911102C069E201C0AB
:1036E00065E3C9010E944C1D0AC080915D028111F1
:1036F00002C069E201C065E3C9010E94571D0E9432
:10370000140D80E001C081E0DF91CF9108950F9307
:103710001F93CF93DF93C42FD22FFC018281882384
:10372000C9F0409360020E94101E90935F02809344
:103730005E0280E28C0F883008F057C0C77081E0CD
:1037400001C0880FCA95EAF7DF91CF911F910F91C1
:103750000C94D70480916002481330C080915E02BF
:1037600090915F020E94281E883C910538F510E276
:103770001D0FCD17B9F080E28C0F883040F4C77070
:1037800081E001C0880FCA95EAF70E94DE04183074
:1037900028F581E09D2F977001C0880F9A95EAF770
:1037A0000E94D704802F0E94CE041830F0F4D77006
:1037B00081E001C0880FDA95EAF70AC080E28C0F39
:1037C000883098F4C77081E001C0880FCA95EAF785
:1037D000DF91CF911F910F910C94DE04802FDF9128
:1037E000CF911F910F910C94CE04DF91CF911F9137
:1037F0000F9108950F939C01CB01243F4CE53407B2
:1038000031F188F4293DFCE53F07D9F02A3D4CE52C
:10381000340779F1283D3C45A9F506E221EE41EE59
:1038200068ED7CE52BC0263FFCE53F07E1F0A8F002
:10383000273F3C4539F507E225EE46EE67EF7CE58C
:103840001DC007E225EE45EE69ED7CE517C006E2F6
:1038500021EE40EE64EF7CE511C007E225EE44EE78
:1038600065EF7CE50BC006E221EE42EE66EF7CE5FB
:1038700005C008E221E045EE6AED7CE50E94871B69
:1038800080E008C0FC018281882319F01092600258
:1038900001C081E00F91089590938F0180938E0174
:1038A000089590936602809365020895E091650201
:1038B000F0916602309721F00190F081E02D09949B
:1038C00080E00895E0916502F0916602309799F0EA
:1038D00020911A01222359F020918E0227FF07C060
:1038E000DC012C9111962C93119726E02C930280E9
:1038F000F381E02D09940895E0916502F09166024C
:10390000309739F022E0DC012C930480F581E02D22
:1039100009940895209163023091640228173907B1
:1039200071F09093640280936302E0916502F091DC
:103930006602309721F00680F781E02D0994089502
:1039400020916102309162022817390771F090933B
:10395000620280936102E0916502F0916602309705
:1039600021F00084F185E02D09940895FC01329640
:1039700080911A01882331F080918E0287FF02C066
:103980009EE101C096E080E0915028F02191222331
:10399000D9F38F5FF9CF0895662351F120911A0171
:1039A0002223E9F020918E0227FF19C0462F469569
:1039B000469546954E31E0F4677021E030E002C054
:1039C000220F331F6A95E2F7FC01E40FF11D82819B
:1039D00090E02823392381E0232B69F409C0FC01FE
:1039E000329608962191621729F0E817F907D1F766
:1039F00080E0089581E008959C01FC0132969FEFDC
:103A000080E04191461789F09F3F19F4411101C0B0
:103A1000982F8F5F8630A9F79F3F39F0F901E90FA2
:103A2000F11D97FDFA956283089508959C012A5F20
:103A30003F4FFC014281461301C01282019682175A
:103A40009307B9F70895262F2695269526952E31AA
:103A500068F4FC01E20FF11D677021E030E001C065
:103A6000220F6A95EAF78281282B22830895262F58
:103A70002695269526952E3170F4FC01E20FF11D56
:103A8000677021E030E001C0220F6A95EAF72095C7
:103A9000828128232283089520911A01222329F06C
:103AA00020918E0227FD0C94231D0C94FC1C209168
:103AB0001A01222329F020918E0227FD0C94371D34
:103AC0000C94161D20911A01FC013296222331F02C
:103AD00080918E0287FF02C08EE101C086E0DF0187
:103AE0001D928A95E9F7089508950C94741D83E05A
:103AF000809367020C94751D811102C081E001C0A2
:103B000082E0809367020C94751D0C947C1D81E00B
:103B1000809367020C94751D0C94871D08950C9476
:103B20008E1D0C948F1D0C948E1D0C948E1D0C9468
:103B30008E1DCF930E94951D0E9473120E94931DAB
:103B4000C0E08C2F0E949D11892B29F4CF5FC430D7
:103B5000C1F780E001C081E0CF91089508951F92E0
:103B60000F920FB60F9211248F939F93AF93BF9331
:103B700080916802811113C08091A1029091A202EC
:103B8000A091A302B091A4024196A11DB11D809302
:103B9000A1029093A202A093A302B093A402BF91AA
:103BA000AF919F918F910F900FBE0F901F9018951E
:103BB0008091A902843031F10E94200310926802A2
:103BC00020E488E190E00FB6F894A8958093600017
:103BD0000FBE2093600083B7817F846083BF83B76B
:103BE000816083BF7894889583B78E7F83BF0FB63B
:103BF000F894A8958091600088618093600010928D
:103C000060000FBE08950E947A070C94270382E09B
:103C100084BD93E095BD9AEF97BD80936E000895A3
:103C20002FB7F8948091A1029091A202A091A302D3
:103C3000B091A4022FBF08952FB7F8946091A1020C
:103C40007091A2028091A3029091A4022FBF0895C7
:103C50009C014FB7F8948091A1029091A202A0918B
:103C6000A302B091A4024FBF821B930B08957894D6
:103C70001F920F920FB60F9211248F939F93AF93C1
:103C8000BF938091A1029091A202A091A302B09152
:103C9000A4020196A11DB11D8093A1029093A202DE
:103CA000A093A302B093A402BF91AF919F918F9173
:103CB0000F900FBE0F901F90189581E08093E00049
:103CC00080E28093D8001092C9008FE19EE40197B2
:103CD000F1F700C0000087E090EBDC018093B202B6
:103CE0009093B302A093B402B093B5029CE088E134
:103CF0000FB6F894A895809360000FBE9093600073
:103D0000FFCF80918C020895089522E02093E9006E
:103D10002FEF3091E800215035FD06C035ED3A9582
:103D2000F1F700002111F5CF2091E80025FF0BC02D
:103D300040E050E066E070E00E94AF208091E80033
:103D40008E778093E8000895CF93DF9320911A0136
:103D5000222339F020918E0227FF03C060E222E087
:103D600002C068E021E02093E9002FEF3091E800E5
:103D7000215035FD06C035ED3A95F1F700002111CF
:103D8000F5CF2091E80025FF1DC0EC0180911A01BC
:103D9000811105C040E050E068E070E003C070E0D1
:103DA00040E050E0CE010E94AF208091E8008E7785
:103DB0008093E80080E2FE01ACE6B2E001900D9253
:103DC0008A95E1F7DF91CF9108958093690270930E
:103DD0006B0260936A028091A902843001F582E04F
:103DE0008093E9008FEF9091E800815095FD06C027
:103DF00095ED9A95F1F700008111F5CF8091E800DB
:103E000085FF0DC040E050E063E070E089E692E09D
:103E10000E94AF208091E8008E778093E80008959B
:103E2000BC0184E00C94E51EBC0183E00C94E51E0B
:103E30000C948C1D6091A50281E0611101C080E0AD
:103E40000C94771D9091A90281E0943009F080E0F4
:103E50006091A5020C947C1D42E061EC81E00E941F
:103E6000B32142E261EC82E00E94B3219091A90269
:103E700081E0943009F080E06091A5020C94851DEA
:103E80008091AB02833009F45DC030F4813071F071
:103E9000823009F496C008958A3009F482C08B30CC
:103EA00009F468C0893009F0A4C020C08091AA023A
:103EB000813A09F09EC08091E800877F8093E800F6
:103EC0008091AE029091AF02892B21F460E28CE6E2
:103ED00092E003C060E080E090E070E00E94FA2091
:103EE0008091E8008B778093E80008958091AA0282
:103EF000813209F07EC08091AE029091AF020297AC
:103F000008F077C08091E800877F8093E800809177
:103F1000E80082FD05C08091A9028111F8CF69C037
:103F20008091F200823031F48091F100813011F003
:103F3000863021F48091F10080938C028091E8001A
:103F40008B7753C08091AA02813A09F052C08091C8
:103F5000AE029091AF02892B09F04BC08091E8002E
:103F6000877F8093E8008091E80080FFFCCF8091FC
:103F70001A0136C08091AA028132D9F58091AE0231
:103F80009091AF02892BA9F58091E800877F8093FB
:103F9000E8000E94E8218091AC0280931A010C9401
:103FA0007A078091AA02813221F58091E800877F0B
:103FB0008093E8000E94E8218091AD0280938D02F9
:103FC00008958091AA02813AA1F48091E800877F48
:103FD0008093E8008091E80080FFFCCF80918D0203
:103FE0008093F1008091E8008E778093E8000C9434
:103FF000E821089584B7877F84BF0FB6F894A89509
:1040000080916000886180936000109260000FBE14
:1040100090E080E80FB6F89480936100909361007F
:104020000FBE0C94871D0E943A220E948D22E2EE60
:10403000F0E080818460808378940C94F1248EE099
:1040400091E00C94511C8091A9028530A9F48091D3
:10405000A902853079F40E94D81D8091A702882397
:10406000B1F30E94991D882391F30E9499200E9428
:104070007A07EDCF0C94031E089508950C94402008
:10408000292F332723303105C9F060F42130310561
:1040900081F02230310509F044C08BE390E02AE042
:1040A00033E043C021323105E1F02232310549F1DC
:1040B00038C082E190E025E433E037C099278130B1
:1040C000910549F028F0029761F5ECECF2E005C0AB
:1040D000E6E0F3E002C0EEEDF2E0849190E09F01B3
:1040E00024C06115710541F061307105D1F489E09A
:1040F00090E025E333E019C089E090E02CE133E063
:1041000014C06115710541F06130710551F486EB01
:1041100090E027E533E009C080E490E02DE034E052
:1041200004C080E090E020E030E0FA013183208399
:10413000089584E089BD86E089BD09B400FEFDCF05
:104140008091D8008F7D8093D8008091E0008260BC
:104150008093E0008091E00081FDFCCF0895CF9234
:10416000DF92EF92FF920F931F93CF93DF93EC01B7
:104170008B017A010E940722811133C0E114F104FE
:1041800039F0F70180819181081B190BC80FD91FE5
:10419000C12CD12C0115110519F18091E80085FD84
:1041A00016C08091E8008E778093E800E114F10456
:1041B00049F0F70180819181C80ED91ED182C08259
:1041C00085E00FC00E940722882321F30AC089914D
:1041D0008093F10001501109FFEFCF1ADF0ADACF07
:1041E00080E0DF91CF911F910F91FF90EF90DF90D2
:1041F000CF9008952091B0023091B1022617370771
:1042000048F06115710539F42091E8002E7720936C
:10421000E80001C0B901FC0120E06115710561F100
:104220008091A9028823D9F18530D9F18091E800E5
:1042300083FD39C08091E80082FD2BC08091E800A9
:1042400080FFEBCF8091F20090E06115710551F095
:104250008830910538F421912093F1006150710963
:104260000196F3CF21E0089709F020E08091E80063
:104270008E778093E800D1CF2111D2CF0AC08091F0
:10428000A902882361F0853061F08091E80083FD08
:104290000AC08091E80082FFF2CF80E0089582E0BA
:1042A000089583E0089581E008952091B00230914F
:1042B000B1022617370748F06115710539F42091CE
:1042C000E8002E772093E80001C0B901FC0120E04E
:1042D0006115710579F18091A902882309F43DC027
:1042E000853009F43CC08091E80083FD3AC080919C
:1042F000E80082FD2CC08091E80080FFE9CF80912A
:10430000F20090E06115710559F08830910540F494
:1043100024912093F1003196615071090196F2CFFA
:1043200021E0089709F020E08091E8008E778093E3
:10433000E800CECF2111CFCF0AC08091A9028823F7
:1043400061F0853061F08091E80083FD0AC08091C2
:10435000E80082FFF2CF80E0089582E0089583E0D4
:10436000089581E00895982F953068F59093E900BD
:10437000981739F07091EC002091ED005091F00009
:1043800003C0242F762F50E021FD02C09F5FECCFA9
:104390003091EB003E7F3093EB003091ED003D7F9C
:1043A0003093ED003091EB0031603093EB0070936F
:1043B000EC002093ED005093F0002091EE0027FDDB
:1043C000E5CF80E008958F708093E90081E0089543
:1043D0008091AA0287FF11C08091E80082FD05C08C
:1043E0008091A9028111F8CF11C08091E8008B77EC
:1043F0000BC08091A902882349F08091E80080FFDA
:10440000F8CF8091E8008E778093E800089520919E
:10441000E4003091E50095E64091EC00842F817036
:1044200040FF23C08091E80080FD1DC08091A9025B
:10443000882399F0853099F08091EB0085FD11C0BB
:104440004091E4005091E5002417350729F391507D
:1044500011F09A01E1CF84E0089582E0089583E0AD
:10446000089581E0089580E008954091E80042FFBA
:10447000DDCF08950E9497220E949A22E0EEF0E09C
:10448000808181608083E8EDF0E080818F77808398
:1044900019BCE3E6F0E08081816080831092A8027D
:1044A00008950E9497220E949A228091D8008F77C7
:1044B0008093D8008091D80080688093D800809144
:1044C000D8008F7D8093D80084E089BD86E089BDC7
:1044D00009B400FEFDCF1092A9021092A50210921D
:1044E000A7021092A60242E060E080E00E94B321A1
:1044F0008091E1008E7F8093E1008091E2008160F5
:104500008093E2008091E20088608093E2008091D5
:10451000E0008E7F8093E0000895E3E6F0E0808184
:104520008E7F808381E08093A8020C9451221092A8
:10453000E20008951092E10008951F920F920FB6C5
:104540000F9211242F933F934F935F936F937F9319
:104550008F939F93AF93BF93EF93FF938091E1006D
:1045600082FF0BC08091E20082FF07C08091E100D2
:104570008B7F8093E1000E94F0248091E10080FF16
:1045800019C08091E20080FF15C08091E2008E7F0B
:104590008093E2008091E20080618093E20080914C
:1045A000D80080628093D80019BC85E08093A9026E
:1045B0000E941A1F8091E10084FF30C08091E200C8
:1045C00084FF2CC084E089BD86E089BD09B400FE6B
:1045D000FDCF8091D8008F7D8093D8008091E1003D
:1045E0008F7E8093E1008091E2008F7E8093E200D5
:1045F0008091E20081608093E2008091A50288238F
:1046000011F084E007C08091E30087FD02C081E0E3
:1046100001C083E08093A9020E94221F8091E100E3
:1046200083FF29C08091E20083FF25C08091E100D3
:10463000877F8093E10082E08093A9021092A50217
:104640008091E1008E7F8093E1008091E2008E7F77
:104650008093E2008091E20080618093E20042E07A
:1046600060E080E00E94B3218091F0008860809338
:10467000F0000E94181FFF91EF91BF91AF919F91A1
:104680008F917F916F915F914F913F912F910F90FB
:104690000FBE0F901F9018951F920F920FB60F929A
:1046A00011242F933F934F935F936F937F938F9337
:1046B0009F93AF93BF93CF93DF93EF93FF93C091FB
:1046C000E900CF708091EC00D82FD17080FDD0E848
:1046D0001092E9008091F000877F8093F000789439
:1046E0000E9490231092E9008091F00088608093EE
:1046F000F000CD2BCF70C093E900FF91EF91DF91D7
:10470000CF91BF91AF919F918F917F916F915F9169
:104710004F913F912F910F900FBE0F901F901895C2
:104720001F93CF93DF93CDB7DEB7AA970FB6F89458
:10473000DEBF0FBECDBFEAEAF2E08091F1008193C7
:1047400022E0E23BF207C9F70E94401F8091E80097
:1047500083FF2EC18091AA029091AB02492F50E0B5
:104760004A30510508F024C1FA01E457FF4F0C9478
:104770008925803821F0823809F01AC108C080915B
:10478000A6029091A702992389F082600FC08091C0
:10479000AE028F70853008F00BC18093E9008091E4
:1047A000EB0085FB882780F91092E9009091E800E2
:1047B000977F9093E8008093F1001092F100D1C0B0
:1047C000282F2D7F09F0F4C0882319F0823061F082
:1047D000EFC08091AC02813009F0EAC0933009F05B
:1047E00080E08093A7022EC08091AC0281112AC084
:1047F0008091AE028F702FEF280F243008F0D8C0C0
:104800008093E9002091EB0020FF1CC0933021F43D
:104810008091EB00806214C09091EB0090619093C6
:10482000EB0021E030E0A90102C0440F551F8A953A
:10483000E2F74093EA001092EA008091EB00886072
:104840008093EB001092E9008091E800877F8093CD
:10485000E8000E94E821ACC08111AAC01091AC020E
:104860001F778091E3008078812B8093E300809113
:10487000E800877F8093E8000E94E8218091E800AB
:1048800080FFFCCF8091E30080688093E3001111EA
:1048900002C082E001C083E08093A90289C08058F1
:1048A000823008F085C08091AC029091AD028C3DC1
:1048B00053E0950779F583E08A838AE289834FB7CD
:1048C000F894DE01139620E03EE051E2E32FF0E0A1
:1048D00050935700E49120FF03C0E295EF703F5FD3
:1048E000EF708E2F90E0EA3010F0C79601C0C096AE
:1048F0008D939D932F5F243149F74FBF8091E8003E
:10490000877F8093E8006AE270E0CE0101960E9402
:10491000FA2016C06091AE027091AF02AE014F5FF7
:104920005F4F0E943E20BC01892B09F441C0909149
:10493000E800977F9093E80089819A810E94552131
:104940008091E8008B778093E80032C0803881F551
:104950008091E800877F8093E8008091A502809392
:10496000F1008091E8008E7772CF811121C0809193
:10497000AC029091AD0299270297D4F48091E8009F
:10498000877F8093E8008091AC028093A5020E940B
:10499000E8218091A502811106C08091E30087FD86
:1049A00002C081E001C084E08093A9020E942C1F14
:1049B0008091E80083FF0AC08091E800877F8093A0
:1049C000E8008091EB0080628093EB00AA960FB61E
:1049D000F894DEBF0FBECDBFDF91CF911F91089538
:1049E0000895CF938091A9028823A1F0C091E90096
:1049F000CF709091EC00892F817090FD80E8C82BDA
:104A00001092E9008091E80083FD0E949023CF700E
:104A1000C093E900CF910895002480FD060E660F33
:104A200011F08695D1F7802D08950024552704C0F4
:104A3000080E591F880F991F009729F076956795E2
:104A4000B8F37105B9F7802D952F0895EE27FF274C
:104A5000AA27BB2708C0A20FB31FE41FF51F220F10
:104A6000331F441F551F969587957795679598F343
:104A70007040A9F7009799F7BD01CF010895AA1BCF
:104A8000BB1B51E107C0AA1FBB1FA617B70710F039
:104A9000A61BB70B881F991F5A95A9F7809590956B
:104AA000BC01CD01089597FB072E16F4009407D0A2
:104AB00077FD09D00E943F2507FC05D03EF4909574
:104AC00081959F4F0895709561957F4F0895A1E25C
:104AD0001A2EAA1BBB1BFD010DC0AA1FBB1FEE1F78
:104AE000FF1FA217B307E407F50720F0A21BB30BC3
:104AF000E40BF50B661F771F881F991F1A9469F73F
:104B000060957095809590959B01AC01BD01CF019A
:104B10000895EE0FFF1F0590F491E02D0994FB011D
:104B2000DC0104C08D910190801921F44150504066
:104B3000C8F7881B990B0895F999FECF92BD81BDE6
:104B4000F89A992780B50895A8E1B0E042E050E0D6
:104B50000C94D025262FF999FECF92BD81BDF89AED
:104B6000019700B4021639F01FBA20BD0FB6F894B1
:104B7000FA9AF99A0FBE08950396272F0E94AB2543
:104B80000E94AA25252F0E94AB25242F0C94AB252B
:104B90000196272F0E94AB250C94AA25DC01CB019E
:104BA000FC01F999FECF06C0F2BDE1BDF89A31963D
:104BB00000B40D9241505040B8F70895F894FFCFDB
:104BC000C8001202280850011E0A14010601811EA5
:104BD000A41E851E141F101F841E01E200E900EAB6
:104BE00000B500B600B700CD008301CC008A019269
:104BF0000194012102230224022502260227022A0F
:104C000002B300B4006F007000818283E200E9000B
:104C1000EA00B500B600B700CD008301CC008A01E0
:104C20009201940121022302240225022602270276
:104C30002A02B300B4006F0070008182836437667B
:0E4C40006736353433323130969365949500E3
:00000001FF
